:03000000020050AB
:0100030032CA
:01000B0032C2
:0100130032BA
:01001B0032B2
:030023000201A92E
:01002B0032A2
:1000500075816078FF7600D8FC75D000C2D3C2D419
:10006000759850758920758DFDD28E7590FF75B08D
:10007000FF9001EB12008BD2BCC299D2AFD2AC750B
:100080001200750F30751030020199E4930200934D
:100090003099FDC299F599A3E493B41BF33099FD0F
:1000A00022A810B83F037510300510E61512050898
:1000B000200116B43A03D20122C202C201C2037562
:1000C000080075130075090022C0E05430B43008F0
:1000D000D0E0C394300200DDD0E0C394372002703A
:1000E00030030412017622A908B90207232323232F
:1000F000F50A22B90307450AF509F50A22B90407EA
:1001000023232323F50B22B90509450BF50B2509FC
:10011000F50922B9060A23232323F50C850B832234
:10012000B9070C450CF50C2509F509850C8222B997
:10013000080723232323F50D22B90912450DF50DD8
:10014000B40104D202D2002509F509D2032201B973
:10015000A908530101B901174511F511C374FF95A1
:100160000904B5110201B9C2AC90022D118B2223F2
:10017000232323F51122A908530101B9011445F0E5
:10018000F0A305132509F509E513B50A0BD202C240
:10019000032223232323F5F022E51260FC11A13072
:1001A00000F72002F4C29021A7C0D0C0E020980D33
:1001B0002099030201DDC299F5990201E6C298E592
:1001C00099A80FB83F03750F30F6050F0512E51219
:1001D000B40F13C2AC90025A118B0201E6751200E3
:1001E000750F30751030D0E0D0D0320C4B495438F8
:1001F0003035312028432920522E4C45544F55523A
:100200004E4555520D0A4C4F4144455220494E54DB
:10021000454C2E4845580D0A524541445920464FF9
:1002200052204C4F4144494E472E2E2E1B434845E9
:10023000434B53554D204552524F522121210D0A17
:100240004C4F4144494E472050524F4752414D4D2B
:100250002041424F525445442E1B4552524F523A70
:100260002046554C4C2052584649464F2121210DDD
:100270000A4C4F4144494E472050524F4752414D3E
:0B0280004D2041424F525445442E1BBC
:00000001FF
